:100026000A0A54657374696E6720334220506F72F2
:100036007420285031322C5031332C5031342C500E
:1000460031352C5031362C50313729202E2E2E00AA
:100056000A5479706520616E79206B657973207416
:100066006F2065786974000A0A54657374696E674F
:1000760020492F4F20506F727420285033372C5050
:1000860031312C50313029202E2E2E000A0A54658B
:100096007374696E6720384220506F727420284D41
:1000A6004350323330303829202E2E2E000A0A547F
:1000B600657374696E6720442F4120284D43503480
:1000C6003932312920636820312C32202E2E2E0021
:1000D6000A0A54657374696E6720434F4D322028AF
:1000E6004D4158333130302D525332333229202E80
:1000F6002E2E000A436F6E6E65637420746F204364
:100106004F4D32202831393230302C4E2C382C319C
:1001160029000A616E642075736520636F6D6D61D9
:100126006E64000A3A303C63723E203D20436865A7
:10013600636B000A3A313C63723E203D2045786984
:1001460074202844656C6179203520536563290A3B
:100156000A005465737420434F4D322028343835D5
:10016600290A004279652021000A0A5465737469D8
:100176006E67204B6579312C4B6579322C5370654F
:10018600616B6572202E2E2E000A4B6579312C4B41
:10019600657932203D2000300031000A0A5465732B
:1001A60074696E6720454570726F6D2032344C431A
:1001B6003034202E2E2E20004572726F72202100C0
:1001C6004F4B000A5479706520616E79206B657912
:1001D6007320000A0A54657374696E67205254438B
:1001E60020445331333037202E2E2E000A54797096
:1001F600652028532920746F207365742074696DF7
:10020600652061742032333A35393A353520323833
:100216002F30322F3034000A6F7220616E79206BD6
:1002260065797320746F20436F6E74696E756520EF
:10023600446973706C6179203A000A74696D6520AF
:1002460025303262783A25303262783A2530326289
:10025600782020646174652025303262782F25303D
:100266003262782F253032627800562D453534209B
:1002760076312E3020285465737420525334383525
:1002860029200D0A000A00562D45353420514320F9
:1002960050726F6772616D2076312E3020283832A9
:1002A6004535344145290A00436865636B73756DAE
:1002B6003D253034582053706565643D25750A0028
:1002C600323030382053696C612052657365617233
:1002D600636820436F2E2C4C74642E000A0A00209B
:1002E600202023232323204D61696E204D656E75E2
:1002F6002023232323200A00312E20334220506F4F
:10030600727420285031322C5031332C5031342C19
:100316005031352C5031362C50313729200A0032D5
:100326002E20492F4F20506F727420285033372CBF
:100336005031312C50313029200A00332E203842DA
:1003460020506F727420284D435032333030382994
:10035600200A00342E20442F4120284D43503439A2
:10036600323129200A00352E20434F4D3220284DA8
:1003760041583331303029200A00362E204B65791A
:100386002C537065616B6572200A00372E20454537
:1003960070726F6D2032344C433034200A00382E90
:1003A6002052544320445331333037200A00202052
:0C03B6002053656C656374203A0007005A
:0411E6007F647E00A4
:1011EA00EF4E60147D527C03ED1D70011CED4C70B6
:0811FA00F7EF1F70EB1E80E807
:0112020022C9
:06093600F553F5527F1E8F
:02093C008F51D9
:10093E00E4FFFEFDFCAB55AA54A953A852D3120AEC
:10094E00075003020A06C2B5755601E556D39551F6
:10095E00504D74FF2555F555E55434FFF554E553C8
:10096E0034FFF553E55234FFF552FCE4FAF9F8E59D
:10097E00552401F555EA3554F554E93553F553E848
:10098E003CF552FC74FF2555F555E55434FFF554EE
:10099E00E55334FFF553EC34FFF552055680ACD2D7
:1009AE00B5755601E556D39551508574FF2555F50D
:1009BE0055E55434FFF554E55334FFF553E5523401
:1009CE00FFF552FCE4FAF9F8E5552401F555EA3540
:1009DE0054F554E93553F553E83CF552FC74FF25B4
:1009EE0055F555E55434FFF554E55334FFF553EC06
:0809FE0034FFF552055680ACF0
:010A060022CD
:100F5400C209E4FFFE7DFF7C1720090B8D828C8380
:100F6400E493F46002D20930090B8D828C83E493FC
:100F74002FFFE43EFEED1D70011CED4C70DB900074
:080F840000E4932FFFE43EFEA0
:010F8C002242
:0E123B00E4FF00000000000000000FBF0AF4F6
:011249002282
:0512BD00D2A602123B65
:0312AE001212BD5C
:0512B100C2A602123B81
:0E125900D2A7D2A6C2A712123BC2A6D2A722CB
:0A127300C2A7D2A612123BD2A72296
:07103200121259AF017E000C
:04103900AB07AA0651
:10103D007D01EB33920AA20A92A7EB25E0FBEA337E
:10104D00FA1212AE0DBD09EAD2A71212BDA2A792D5
:06105D000A1212B1A20A02
:01106300226A
:10119F00E4FE7D011212BDA2A7920AEE25E0FEA287
:1011AF000AE43342061212B10DBD09E8D2A712129A
:0311BF00AEAF06CA
:0111C200220A
:10114E00E4FE7D011212BDA2A79209EE25E0FEA2D9
:10115E0009E43342061212B10DBD09E8C2A71212FC
:08116E00BD1212B1D2A7AF06B9
:011176002256
:060FC6008E4D8F4EAC05BC
:100FCC00E54E7807CEC313CE13D8F9540E44A0FEC9
:100FDC00121259AF067E00121039AF4EAE4D1210E0
:100FEC0039AF047E001210391212737F050211EA18
:040E97008E4D8F4E9F
:100E9B00E54E7807CEC313CE13D8F9540E44A0F900
:100EAB00121259E9FF7E00121039AF4EAE4D1210DF
:100EBB00391212737F017E001211EA4301011210E5
:0B0ECB003212119FAE07121273AF0627
:010ED60022F9
:0A127D00532E7F5330BF5335EC228F
:1011C3001212597FD07E00121039E4FF121039E455
:1011D300FC742E2CF8E6FF7E001210390CBC08F1CB
:0311E30002127382
:100FFC001212597FD07E00121039E4FF12103912F0
:10100C00127312123B1212597FD1121039E4FC12D6
:10101C00114EA907742E2CF8A6010CBC07F1121165
:06102C009F8F35021273D4
:0B106400E54FFB7A007D0A7C00E4FFF2
:10106F008C508D51A9078B828A83E925E0540E4459
:10107F0040F9121032AF51AE50121039AF82AE8319
:06108F0012103902127379
:1010F400430630C2A2C2A3E4FDEE30E704D2A080CE
:1011040002C2A0EF25E0FFEE33FE0000D2A20000F1
:0C1114000000C2A200000DBD10DFD2A33D
:0111200022AC
:10112100430630C2A2C2A4E4FDEE30E704D2A0809F
:1011310002C2A0EF25E0FFEE33FE0000D2A20000C4
:0C1141000000C2A200000DBD10DFD2A40F
:01114D00227F
:040F1700AD07AC0670
:100F1B00E4FBFAD2A1C2A2C2A5F9EC30E704D2A03D
:100F2B008002C2A0ED25E0FDEC33FCD2A20000EB69
:100F3B0025E0FBEA33FA30A103430301C2A209B94E
:080F4B0010D8D2A5AE02AF03DD
:010F5300227B
:0712B6007F097EC0020F1743
:021203008F4F0B
:101205007F007E40120F17EE30E6F5AF4F7480FE7B
:03121500020F17AE
:1010C500E4F54E7437254EF8E6FF6022EFAF4EB4D7
:1010D5000A0F054E74372FF8E6FF1212037F0D80B5
:0E10E50008054E74372FF8E6FF12120380D56F
:0110F30022DA
:101218007F007E40120F17EE30E7F5E4FFFE120F55
:0112280017AE
:0112290022A2
:10071E00758910E4F58DF58BC28E20B0FDD28EA2B8
:10072E00B0B340FBC28EAF8DAB07EBFAAF8BEFFBD6
:10073E00E47F64FE1211EA7F20D3EB94E4EA941175
:10074E00400AEB940CEA941250028060D3EB94E8CA
:10075E00EA9408400AEB9410EA940950028065D39B
:10076E00EB946AEA9404400AEB9492EA94045002E1
:10077E00806AD3EB942CEA9402400AEB9454EA94E8
:10078E00025002806FD3EB940CEA9401400BEB9471
:10079E0034EA9401500302082B7F3AD3EB94EAEA31
:1007AE009405400FEB9412EA94065007752C0475CD
:1007BE002DB022D3EB94ECEA9402400FEB9414EAA2
:1007CE0094035007752C09752D6022D3EB946CEAB7
:1007DE009401400FEB9494EA94015007752C127516
:1007EE002DC022D3EB94ACEA9400400FEB94D4EAE4
:1007FE0094005007752C25752D8022D3EB944CEA6E
:10080E00940040047E0180027E00C3EB9474EA944F
:10081E000050047D0180027D00ED5E6007752C4B5B
:0A082E00752D00221211E602071ECC
:100E5400759852758920E52D852CF0120A1D0E7A9D
:100E640004B00E7F09600E8412C00E8925800E8E98
:100E74004B0000000E94758DE88015758DF480107C
:100E8400758DFA800B758DFD8006758DFD43878009
:030E9400D28E22D9
:0E124A0012129BAB077F0A7E001211EAAF035F
:011258002273
:0A1287007F057E001211EAD2B422A6
:0A1291003014FD00000000C2B4227A
:100ED700BF3A0FE4F536D2167E097823E4F608DE2A
:100EE700FC2230162AEF640D6003BFFF0C74232524
:100EF70036F8A607C216D21322EFC394204010E596
:0F0F070036C39408500974232536F8A60705361B
:010F160022B8
:0300230002117750
:0D117700C0E0C0D075D000C000C006C007A9
:10118400309906C299D2148007AF99C298120ED72B
:0B119400D007D006D000D0D0D0E03251
:100003003015093014FDC2148F998012BF0A0830CD
:0F00130099FDC29975990D3099FDC2998F992267
:100E0D007BFF7A0079261204247BFF7A0079561233
:100E1D000424E4FB2098208B20A2009292A2019240
:100E2D0093A2029294A2039295A2049296A2059285
:100E3D00971211E60B80DD12124AD292D293D29400
:060E4D00D295D296D29767
:010E5300227C
:100F8D007BFF7A00796D1204247BFF7A007956126B
:100F9D000424E4FB2098188B20A20092B7A20192A2
:100FAD0091A20292907F2C7E011211EA0B80E51224
:080FBD00124AD2B7D291D29082
:010FC5002209
:100C73007BFF7A007992120424E4FBFA7D0AFCFFDD
:100C830012106FE4FBFAFDFF12106F754E01754FE2
:100C930001754D011210647F2C7E011211EAE54F9C
:100CA30025E0F54F054DE54DD3940840E7054EE5A6
:100CB3004ED3940340D8754D01754F551210647F80
:100CC300E87E031211EA754FAA1210647FE87E03CF
:100CD3001211EA054DE54DD3940340DDE4F54FE5EC
:0D0CE3004FFB7A007D0A7C00E4FF02106FD9
:100CF0007BFF7A0079B31204247BFF7A00795612C5
:100D00000424E4FBFA803B20983DAF03AE021210AE
:100D1000F4AF82AE831211217F027E001211EA0B22
:100D2000BB00010AD3EB94FFEA940F4003E4FAFB03
:100D3000E582158270021583E582B4FFCAE583B4AB
:100D4000FFC5900FFF80C0E4FFFE1210F4E4FFFE29
:060D500012112102124AFB
:100AD8007BFF7A0079D61204247BFF7A0079F91219
:100AE80004247BFF7A0179181204247BFF7A0179A8
:100AF800291204247BFF7A0179391204241212B6D0
:100B0800C209200915121218BF3AF71212188F4D90
:100B1800121218BF0DECD20980E8E54DB4301E75ED
:100B280054FF7555017556587B007A0079371204C1
:100B38001E1210C57F327E001211EA80C3E54DB443
:100B480031BE7554FF7555017556697B007A007979
:0E0B58003712041E1210C57F887E131211EA98
:010B6600226C
:100BF2007BFF7A01796F1204247BFF7A0079561207
:100C02000424754EFF209866E4F54D30B303434D3E
:100C12000230B203434D01E54D654E60E8E475557F
:100C220010755427120936E4755510755427F5537B
:100C3200F5527F1412093C7BFF7A01798F1204244A
:100C4200854D4FE4F550E54F7BFF20E0067A0179B0
:100C52009D80047A01799F120424E54FC313F54F56
:100C62000550E550D3940140DD854D4E8097021228
:010C72004A37
:100DB8007BFF7A0179A11204247DAAE4FFFE120FB9
:100DC800C67D557F017E00120FC6C209E4FFFE12E0
:100DD8000E97EF64AA6002D2097F017E00120E9777
:100DE800EF64556002D2097BFF3009067A0179BEAB
:100DF80080047A0179C61204247BFF7A0179C9122A
:050E0800042402124A5F
:100B67007BFF7A0179D91204247BFF7A0179F2128B
:100B770004247BFF7A02791D12042412124A8F4D36
:100B8700E54D64536005E54DB4732275322875331E
:100B970002753404753101753023752F59752E553B
:100BA70012127D1211C37FC87E001211EA7BFF7AF1
:100BB700007956120424754DFF20982C1211E61265
:100BC7000FFCE52E654D60F17BFF7A027940853099
:100BD70054852F55852E5685325785335885345978
:0B0BE700120424852E4D80D102124A1A
:0912A5007BFF7A02797002042437
:10109500D215D2ACD2AFE4F536D2167F097823E467
:1010A500F608DFFC7F093013FDC213121287AF2348
:1010B50012122AEF24D070031212A512129180E6A3
:100D5600E475552075544E120936C2B4D29912075D
:100D66001E120E54BF3A03121095C21512128712A4
:100D76000F548E4E8F4F754D017BFF7A02798B1281
:100D86000424054DE54DD3941640EE7BFF7A027997
:100D96008D1204247BFF7A0279AE854E54854F5519
:100DA600852C56852D571204247BFF7A0279C602BC
:020DB600042413
:10083800E4F54B120D56D2083008637BFF7A027933
:10084800E21204247BFF7A0279E51204247BFF7A02
:100858000279FE1204247BFF7A0379251204247B93
:10086800FF7A0379411204247BFF7A037959120431
:10087800247BFF7A03796C1204247BFF7A03798046
:100888001204247BFF7A0379911204247BFF7A03F4
:1008980079A41204247BFF7A0379B4120424C208D1
:1008A800E54B6007F54CE4F54B800812124A12122A
:1008B8002A8F4CE54C24CFB4080050669008D275B6
:1008C800F003A4C58325F0C583730208EA0208F281
:1008D8000208FA02090202090A02091202091A02A6
:1008E8000922D208120E0D020840D208120F8D02FA
:1008F8000840D208120C73020840D208120CF00209
:100908000840D208120AD8020840D208120BF20294
:100918000840D208120DB8020840D208120B67022C
:0E09280008407BFF7A0379C0120424020840C5
:0300000002126782
:0C126700787FE4F6D8FD75816402083839
:100A0700EB9FF5F0EA9E42F0E99D42F0EC6480C866
:060A170064809845F02206
:100A1D00D083D082F8E4937012740193700DA3A368
:100A2D0093F8740193F5828883E473740293B5F09F
:0D0A3D00067403936860E9A3A3A3A380D807
:1003C200E5602454F8E60560227851301102785431
:1003D200E475F001120AA2020A4A200AEB7F2ED229
:1003E2000A8018EF540F2490D43440D4FF300E0BFF
:1003F200EF24BFB41A0050032461FFE561600215C7
:10040200610564E5647002056330110D7851E4758D
:10041200F001120AA2EF020A900200037403D21141
:100422008003E4C211F5608B518A528953E4F5616D
:10043200F563F564E56160077F201203FD80F575C1
:1004420062FFC20BC20AC20CC20DC20FC210C2129C
:100452001203CBFF700D3011057F0012040EAF6442
:10046200AE6322B4255FC2D5C20E1203CBFF24D0E5
:10047200B40A00501A75F00A786130D50508B6FF43
:100482000106C6A426F620D5047002D20D80D92416
:10049200CFB41A00EF5004C2E5D20E02060ED20B00
:1004A20080C6D20A80C0D20C80BCD2D580BAD20F0C
:1004B20080B47F201203FD200C077401B561004057
:1004C200F11203C2FF1203FD020436D212D21080CF
:1004D200951203C2FB1203C2FA1203C2F94A4B700D
:1004E2000679DF7A067BFF200C2EE561602A7E000A
:1004F2008E82758300120A6360060EEE656270F0EA
:10050200C2D5EBC0E0EAC0E0E9C0E0EE120655D089
:10051200E0F9D0E0FAD0E0FB120A4AFF60AAEBC091
:10052200E0EAC0E0E9C0E01203FDD0E02401F9D026
:10053200E03400FAD0E0FBE5620460DCD562D980E9
:10054200877BFF7A067951D20C809C7910800279E0
:1005520008C210C2128008D2D5790A8004790AC270
:10056200D5E562047002F562E4FAFDFEFF1203C2F1
:10057200FC7B08200B131203C2FD7B10300A0A1207
:1005820003C2FE1203C2FF7B20EC3382D592D55008
:1005920013C3E4300A069FFFE49EFEE4200B039D92
:1005A200FDE49CFCE4CBF8C20BEC700CCFCECDCCBE
:1005B200E824F8F870F38017C3EF33FFEE33FEED53
:1005C20033FDEC33FCEB33FB994002FB0FD8E9EB34
:1005D200300B05F8D0E0C448B20BC0E00AEC4D4E37
:1005E2004F78207B0070C2EAB5620040BCC0E012C6
:1005F2000657D0F0D0E0200B04C4C0E0C4B20BC058
:10060200F01203E6D0F0D5F0EB020436120AB2047F
:10061200D353054D5804A44C04A04205514F05592B
:0F0622004405594904B943055F5505434605434F
:100631004505434706FF5004A82D04AC2E04CF2BDB
:1006410004B02304CD2006E82A046848000004C74A
:100651003F3F3F00790AA2D5200D14300F09B91090
:10066100020404B9080104A2D5201002500104209B
:100671000C68920CB561005034C0E07F20300D1938
:100681007F30A20C7210720F500F1206AEC20CC254
:1006910010C20FC2127F30800F300F03E9C0E01289
:1006A10003FD300F03D0E0F9D0E0B561CC300F1776
:1006B1007F30B9100C1203FD7F58300E077F788010
:1006C10003B908031203FD300C057F2D0203FD7FE2
:1006D100202012F87F2B2010F322920C80CF286E5D
:1006E100756C6C2900D20B1203C2300BF8C20B7867
:1006F1006130D50108F60204682D504349581203B0
:10070100C22403B405004001E49006FA931203EEFB
:0D071100743A1203EED20D75610402054D1D
:0A129B003098FDAF99C2987E002242
:10122A00EFC39461400AEF947B5005EF24E0FF225C
:01123A002291
:100A4A00BB010689828A83E0225002E722BBFE02AA
:090A5A00E32289828A83E49322DD
:100A6300BB010CE58229F582E5833AF583E0225048
:100A730006E92582F8E622BBFE06E92582F8E22292
:0D0A8300E58229F582E5833AF583E49322AC
:100A9000BB010689828A83F0225002F722BBFE0145
:020AA000F3223F
:100AA200FAE6FB0808E6F925F0F618E6CA3AF62255
:100AB200D083D082F8E4937012740193700DA3A3D3
:100AC20093F8740193F5828883E4737402936860E7
:060AD200EFA3A3A380DFE7
:00000001FF
